:1000000000308A001E2D00000A108A100A11820793
:100010003E347F34713459344D347F343E3440346F
:1000200042347F347F34403440340034623473349B
:10003000593449346F3466340034223463344934DB
:1000400049347F343634003418341C341634533475
:100050007F347F34503427346734453445347D341D
:10006000393400343C347E344B34493479343034C0
:10007000003403340334713479340F3407340034DA
:1000800036347F34493449347F34363400340634CE
:100090004F34493469343F341E3400341C343E3408
:1000A00063344134413463342234083408343E34F8
:1000B0003E34083408340034083408340834083432
:1000C00008340834003400340034603460340034C0
:1000D0000034003400340034063409340934063462
:1000E0000034003400340034003400340034003470
:1000F0000A108A100A11820700348034C034E034B8
:10010000F034F834FC34FE34FF34FF348316010835
:10011000C73908388100831290019A01073099008D
:100120008316050803308312A000A00B9528190838
:100130008C11831699010C3085008312452D7D307A
:10014000840000080319B2280130A100A001A00B0F
:10015000A728A10BA6284A30A000A00BAD28B028E4
:10016000800BA428003408308316A000A0080319CF
:10017000D2288512831285127F088039031DC52875
:100180008316051283120512C928831605128312DD
:10019000051683168512831285160310FF0D83162C
:1001A000A003B628831200348316051083120510AD
:1001B0007E08FF00B32000347C0807394038FD007A
:1001C000FE00D4207B087F398038FD00FE00D4205B
:1001D000003483160510831205147B08FF00B3203A
:1001E00000348316051083120514831685108312BC
:1001F00085106430FD009F208316851083128514BE
:100200002130FE00D420C830FE00D4201330FE0080
:10021000D4202030FE00D4200930FE00D420FB0181
:10022000FC01DC200130F500F830F400F408031D77
:100230001C29F50803192329FB01E9207408031977
:10024000F503F40316290830FE00D4200C30FE001C
:10025000D420FB01FC01DC20462D7508FB0076084C
:10026000FC00DC207708F90078087707790203188A
:100270004629790883169B009C131C141A08FA005F
:100280007A08FB008312E920F90A3429003440304F
:10029000F500F601F7011330F8002D214030F5008C
:1002A0000130F6001330F700F8002D214030F50042
:1002B0000230F6002630F7001330F8002D214A30C6
:1002C000F5000330F6003930F7000930F8002D2131
:1002D0004830F5000430F6004230F7000930F800ED
:1002E0002D210230F5000530F6004B30F70050307C
:1002F000F8002D21FB010130FC00DC20FF30FB0069
:10030000E920F4017408383C031C8B290130FB0000
:10031000E920F40A82294330FB00E920FF30FB008A
:10032000E920FB010230FC00DC20FF30FB00E9206B
:100330003A30FB000230FC00DC200830FB00E920F2
:10034000FF30FB00E920FB010330FC00DC20FF3024
:10035000FB00E920F40174081B3C031CB629FB01D7
:10036000E9202030FB00E920F40AAB29FB01E92059
:100370002130FB00E920FF30FB00E920FB01E920F0
:100380003030FB00E9204830FB00E9204830FB001A
:10039000E9203030FB00E920FB010430FC00DC20C8
:1003A0003F30FB00E920F4017408383C031CDD29D0
:1003B0002030FB00E920F40AD4292430FB00E92096
:1003C0003F30FB00E920672D8316051183120511CC
:1003D000A630A000A00BEA29000083160515A63060
:1003E0008312A000A00BF2290000831605158312CA
:1003F0000034FE017E08073C031C182A83160511F1
:1004000083120511032A0310FD0C0318092A051194
:100410000A2A05158316051113308312A000A00BBC
:100420000F2A122A83160515152AFE0A8312FA29A5
:100430000034FD017D08073C031C3B2A831605118F
:1004400083120511232A8316051502308312A0009A
:10045000A00B282A00008316051583120519322ADD
:100460000310332A0314FE0C2730A000A00B362AF9
:10047000392AFD0A1A2A7E08A1000034A001A10130
:10048000760803107718A007A00CA10CF718A00796
:10049000A00CA10C7719A007A00CA10CF719A007BC
:1004A000A00CA10C771AA007A00CA10CF71AA007AA
:1004B000A00CA10C771BA007A00CA10CF71BA00798
:1004C000A00CA10C0034F5017508063C031C752A2C
:1004D0007408F6000730F7003E2275082107042053
:1004E000F800FB00E920F50A642A0034A101A2010A
:1004F000A001A3017708031D802A760803199A2A10
:100500001030F8000310F40DF50DA00DA30D7708C1
:100510002302031D8D2A76082002031C962A7608E2
:10052000A002031CA3037708A3020314A10DA20DCC
:10053000F80B822A0034F401E421CC30FD00F921CB
:100540004430FD00F921F408031DAA2A19222108CC
:10055000F400A32AE421CC30FD00F921BE30FD00D7
:10056000F92119222108F50019222108F600760840
:10057000F8007508F7007808FE007708FD008E3057
:10058000A0007E08A1007D08A200A301FE1FCD2AC5
:10059000A109A209A20A0319A10AA108031DDA2AC6
:1005A0002208A100A2010830A002A108031DDA2A36
:1005B000A001E32A0310A11BE12AA20DA10DA003B3
:1005C000DA2AFE1FA1132308FC002208FB002108E1
:1005D000FA002008F900C830FD009F207908A0002B
:1005E0007A08A1007B08A2007C08A3002308F7007A
:1005F0002208F6002108F5002008F4008E30A00043
:100600007408A0027508A2007608A100A217A0082D
:100610000319152B0310A208031D112BA1080319A0
:10062000152BA20CA10CA00B0A2BF51F1C2BA1094A
:10063000A209A10A0319A20A2208AC002108AB00F2
:10064000AA010430FB000330FC00DC202C08003C35
:10065000031C312BAC012B1C2F2B0130AA00B00145
:10066000462B0C30F4006322AC012B08003CAB009D
:100670002C08031C2C0F3E2B01303F2B013CAC00FF
:100680002B1C442B0130AA000130B0000310AC0C2D
:10069000AB0C2B08F0002C08F5002B08F400F70138
:1006A0006430F60076222108AD002D08F600643093
:1006B000F7003E222108AB020030031C0130AC02DF
:1006C0002C08F5002B08F400F7010A30F60076221A
:1006D0002108AE002E08F6000A30F7003E2221085D
:1006E000AB020030031C0130AC022B08AF00AD0898
:1006F000031D812B0F30AD00AE08031D812B0F3081
:10070000AE00742D4C30FB00FC01DC200430FB00FB
:10071000E9204C30FB000130FC00DC20FB01E9202B
:100720004C30FB000230FC00DC20FB01E9204C30A7
:10073000FB000330FC00DC20FB01E9202E080F3C0D
:10074000031DAD2B4C30FB000330FC00DC202F08D8
:100750007820F400FB00E9202E2C2E0BC22B4C300D
:10076000FB000330FC00DC20FF30FB00E9204C30B4
:10077000FB000230FC00DC202F087820F400FB0096
:10078000E9202E2C2E08023C031DE12B4C30FB00EF
:100790000330FC00DC20FF30FB00E9204C30FB0084
:1007A0000230FC00DC20FF30FB00E9204C30FB0075
:1007B0000130FC00DC202F087820F400FB00E92049
:1007C0002E2C2E08033C031D0F2C4C30FB00033055
:1007D000FC00DC20FF30FB00E9204C30FB00023045
:1007E000FC00DC20FF30FB00E9204C30FB00013036
:1007F000FC00DC20FF30FB00E9204C30FB00FC015A
:10080000DC202F08053C031C0B2C2F087820F4005B
:10081000FB00E9200E2CF830FB00E9202E2C4C3098
:10082000FB000330FC00DC20FF30FB00E9204C30F3
:10083000FB000230FC00DC20FF30FB00E9204C30E4
:10084000FB000130FC00DC20FF30FB00E9204C30D5
:10085000FB00FC01DC20F830FB00E920D82DF4017E
:100860007408383C031C432C35307407F900013000
:100870007407353E84000008FB00790884007B087B
:100880008000F40A302CB008031D502C70082A3C5C
:10089000031C4D2C7008EE004F2C2A30EE005C2C0F
:1008A000300B5C2C70080E3C031C5A2C70088038EE
:1008B000EE005C2C8E30EE00F4017408383C031C12
:1008C0001D2D3530740784000008F50075087F3C45
:1008D000031C8A2C0310750CF800A0307807F9006F
:1008E0002130FA000318FA0A790883169B009C133A
:1008F0001C141A08F700B6307807F9002130FA0006
:100900000318FA0A79089B009C131C141A08F600B5
:10091000AA2C83128030F5020310750CF800D03039
:100920007807F9002130FA000318FA0A79088316CB
:100930009B009C131C141A08F700D7307807F900A5
:100940002130FA000318FA0A79089B009C131C1442
:100950001A08F600770FAD2C1A2D760BBC2C01303F
:100960007407F900FB007608FC008312DC2077088E
:10097000FB00E920C72C831601307407F900FB0047
:100980000130FC008312DC200130FB00E9207608F6
:10099000023C031DD62C01307407F900FB007608D9
:1009A000FC00DC207708FB00E920DF2C0130740715
:1009B000F900FB000230FC00DC20FB01E920760896
:1009C000033C031DF12C741CE62CF7160130740750
:1009D000F900FB007608FC00DC207708FB00E9202A
:1009E000002D01307407F900FB000330FC00DC200F
:1009F000741CFE2C2030FB00E920002DFB01E920B7
:100A00007608043C031D0F2D01307407F900FB002C
:100A10007608FC00DC207708FB00E920192D013066
:100A20007407F900FB000430FC00DC202030FB00E0
:100A3000E9208316F40A83125D2CDD2D03081F398B
:100A400083005F30A0002130840083138001840A7A
:100A5000A00B262D2030A000A0308400831380013D
:100A6000840AA00B2F2DA00184011F308305613063
:100A700083168F0083121F13003083169100831298
:100A80009A0107309900A5018628F128FE308316C7
:100A90009B009C131C141A088312B300FF308316AA
:100AA0009B009C131C141A088312B4003308B20074
:100AB0003408B100F1017108393C031C662D353052
:100AC00071078400FF308000F10A5B2D4729F30194
:100AD000F20173083202031CDC2D031D732D310853
:100AE00072020318DC2D9B2AB008031D992D3D309E
:100AF000FB00FC01DC20FB01E920FB01E9203D308B
:100B0000FB000130FC00DC20FB01E920FB01E920B7
:100B10003D30FB000230FC00DC20FB01E920FB0142
:100B2000E9200130FB00FC01DC202D08F4006322E9
:100B3000C02D3D30FB00FC01DC200830FB00E9202B
:100B40000830FB00E9203D30FB000130FC00DC20D8
:100B50000830FB00E9200830FB00E9203D30FB00B5
:100B60000230FC00DC200830FB00E9200830FB00EC
:100B7000E9200130FB00FC01DC200C30F400632292
:100B80002E08F40063222F08F40063220D30F400D5
:100B900063222A0BCF2D0530F4006322D12DF401FE
:100BA00063220E30F40063220A30F4006322822BA9
:0E0BB000F20A0319F30A692D2F2C672D63003A
:104200009400A200AA00940080009C00A200A200DA
:104210009C000000F800040004000400F800000006
:10422000000080008000A400B200AA00A40080006A
:104230009C00A200A2009C000000FF000000000003
:104240000000FF0000000800800080008000800067
:104250008400BE0080009C00A200A2009C00000020
:10426000FF00000000000000FF00000008008000C8
:104270008000FF00800080008000FF000000080038
:10428000800080000E001F003F003F002F002F0025
:1042900031001F000E00FE00120012003200CC00A0
:1042A0000000C800A800A800F80000000000FE0000
:1042B0008200820082007C000000FA000000000002
:1042C000FE001000280044008200C800A800A800DA
:1042D000F8000000FE0000000000FE0082008200E6
:1042E00082007C0000007000A800A800B000000060
:1042F00000004C009200920064000000FA000000F0
:1043000000007C0082008200920074000000000027
:1043100080000000700088008800500000007000DD
:104320008800880070000000F80008000800F8000D
:0643300008000800F00087
:10434000200010000800040002000100800040006E
:10435000200010000800040002000100810041005C
:104360002100110009000500030002000300030002
:104370000300030003000300020002000200020029
:104380000200020002000200010001000100010021
:08439000010001000100010021
:1043A000400080002100220024002800300003008B
:0C43B000030004000400040004000400EA
:0443FC000300540066
:02400E00C43FAD
:00000001FF
